:10000000FF3091009200920B0328910B0328860188
:10001000850183169B308600F73085008312861297
:10002000AB208616AB20861C1328AB200611AB2014
:100030008C018D018E01482048204820482048200E
:10004000482048208C0048208C0D0C108C0448203F
:100050008D0D0D108D0448208D0D0D108D04482040
:100060008D0D0D108D0448208D0D0D108D04482030
:100070008E0D0E108E0448208E0D0E108E0448201A
:100080008E0D0E108E0448208E0D0E108E045E28EC
:100090000F309000900B4A2806130F309000900B01
:1000A0004F28061700000000000006089500950C78
:1000B000950C950C950C1508013908000615AB2018
:1000C00030308E078D078C076528253093007B2004
:1000D0000C0893007B200D0893007B200E089300F2
:1000E0007B202F3093007B20373093007B200D3016
:1000F00093007B200F28A020131CA0201318A320FE
:10010000931CA0209318A320131DA0201319A32033
:10011000931DA0209319A320131EA020131AA3201F
:10012000931EA020931AA320131FA020131BA3200B
:10013000931FA020931BA320A020A320A32008008E
:100140008511A62008008515A6200800ED30940032
:10015000940BA82808000F308F00A6208F0BAD2825
:02016000080095
:00000001FF
